:1000000045C0000058C0000056C0000054C00000A9
:1000100052C0000050C000004EC000004CC00000A4
:100020004AC0000048C0000046C0000044C00000B4
:1000300042C0000040C000003EC000003CC00000C4
:100040003AC0000038C0000036C0000034C00000D4
:1000500032C0000030C000002EC000002CC00000E4
:100060002AC0000028C0000026C0000024C00000F4
:1000700022C0000020C000001EC000001CC0000004
:100080001AC0000018C0000016C0000011241FBED6
:10009000CFEFD0E4DEBFCDBF11E0A0E0B1E0E8E8F3
:1000A000FEE000E00BBF02C007900D92A230B10746
:1000B000D9F70BD1E7C6A4CFBF92CF92DF92D90177
:1000C000E6E4F0EF0F921F92D72EC62EB82E242F03
:1000D0001B2E0A2E09952131F9F71F900F90DF9002
:1000E000CF90BF900895BF92CF92DF92D901E6E4FE
:1000F000FEEF0F921F92D72EC62EB82E242F1B2E46
:100100000A2E09952131F9F71F900F90DF90CF90BB
:10011000BF9008950F931F93CF93DF93EC01890154
:10012000CA01DB019C01AD0160E070E00DC04BBF76
:10013000F9018791FE01E60FF71F80832F5F3F4F84
:100140004F4F5F4F6F5F7F4F6017710780F3CE0196
:10015000DF91CF911F910F910895EF92FF920F932E
:100160001F93CF93DF937B018C01BA01E90181E0FA
:100170002130380710F0C0E0D1E080E09FEFAFEF12
:10018000BFEFE822F9220A231B23CB01B801A70104
:100190009E01C0DFCE01DF91CF911F910F91FF90A3
:1001A000EF9008952F923F924F925F926F927F92BD
:1001B0008F929F92AF92BF92CF92DF92EF92FF9277
:1001C0000F931F93CF93DF936B017C01BA0128013A
:1001D000490181E02130380718F0812C91E0992EF7
:1001E00014013694279480E09FEFAFEFBFEF8C218E
:1001F0009D21AE21BF215C016D01CB013B01B60108
:10020000A501EC0110E000E0A0E0B0E018C06BBF79
:10021000FA0127913691888199812817390709F0C9
:1002200011E080959095282B392B2F5F3F4F09F0D7
:1002300001E04E5F5F4F6F4F7F4F11962296A215E0
:10024000B30528F3112319F4882499242AC0002324
:1002500039F0C601B50143E020E030E0F201099534
:1002600086017501C0E0D0E012C0D3012D913D910F
:100270003D01C801B70141E0F201099582E090E03B
:10028000A0E0B0E0E80EF91E0A1F1B1F2196C21560
:10029000D30558F3C601B50145E020E030E0F20196
:1002A0000995C401DF91CF911F910F91FF90EF90BD
:1002B000DF90CF90BF90AF909F908F907F906F9086
:1002C0005F904F903F902F900895CF92DF92EF92E2
:1002D000FF920F931F93DF93CF93CDB7DEB7C0503C
:1002E000D1400FB6F894DEBF0FBECDBF14BE88E17B
:1002F0000FB6F89480936000109260000FBEF894DF
:100300001982009100011091010140E050EE61E07E
:1003100070E0C801AA2797FDA095BA2FABBFFC01DA
:10032000879196916BBFFA012791369182179307B7
:1003300019F081E089830EC00E5F1F4F4E5F5F4F43
:100340006F4F7F4F483A89EE580781E0680780E099
:100350007807F9F68981882309F4A7C03CE8C32E01
:1003600030EED32E31E0E32EF12CC701B6018E0121
:100370000F5F1F4FA80120E031E0EFDE9C0184E712
:100380009BE1A0E0B0E0C80ED91EEA1EFB1EC7012B
:10039000B601A8010CE510E005DF8CE895EEAFEFA3
:1003A000BFEFC80ED91EEA1EFB1E9CE8C91694EECC
:1003B000D90691E0E90690E0F906B9F6EE24FF24AB
:1003C000CE0101966FEF70E040E051E054D580918E
:1003D0000001909101018E0D9F1DAC01662757FD14
:1003E0006095762F28EA39E02E193F09A1E02130E7
:1003F0003A0710F020E031E08E010F5F1F4FC80177
:1004000089DEB70180E090E0605070428E4F9F4FD0
:10041000A80120E031E003E710E0C4DEB0E0EB1615
:10042000B5E0FB0629F080E091E0E80EF91EC8CFA8
:1004300028EAC22E24E0D22ECE0101966FEF70E0A2
:1004400040E051E018D580910001909101018E0D9E
:100450009F1DAC01662757FD6095762F960191E0B0
:10046000C91691E0D90610F020E031E08E010F5F4F
:100470001F4FC8014FDEB70180E090E0605070422E
:100480008E4F9F4FA80120E031E00CE510E08ADE9E
:10049000A0E0B1E0EA0EFB1E80E09FEFC80ED91E7F
:1004A00098EAE91699E0F90638F280E090E0C05049
:1004B000DF4F0FB6F894DEBF0FBECDBFCF91DF91F7
:1004C0001F910F91FF90EF90DF90CF9008957EC025
:1004D0000000BFC00000A3C00000A1C000009FC07A
:1004E00000009DC000009BC0000099C0000097C0A4
:1004F000000095C0000093C0000091C000008FC0B4
:1005000000008DC000008BC0000089C0000087C0C3
:10051000000085C0000083C0000081C000007FC0D3
:1005200000007DC000007BC0000079C0000077C0E3
:10053000000075C0000073C0000071C000006FC0F3
:1005400000006DC000006BC0000069C0000067C003
:10055000000065C0000063C00000BBBEEC2DFD2D97
:10056000B7B6B0FCFDCF27BFE895B7B6B0FCFDCF5E
:1005700021E1B7B6B6FCF4CF0895040309041C03C7
:100580007700770077002E00660069007300630033
:1005900068006C002E00640065000E0355005300D7
:1005A000420061007300700012011001FF0000089A
:1005B000C016DC050201010200010902120001015E
:1005C00000803209040000000000000011241FBE5A
:1005D000CFEFD0E4DEBFCDBF34B7D0E4CEEF29916A
:1005E000203F299109F02FEF20933F0130934001E4
:1005F00011E0A0E0B1E0E2EAF9EE01E00BBF02C0D9
:1006000007900D92A630B107D9F711E0A6E0B1E04E
:1006100001C01D92AF33B107E1F79FD127C457CF77
:10062000A82FB92F80E090E041E050EA609530E0DB
:1006300009C02D9182279795879510F084279527DB
:10064000305EC8F36F5FA8F30895EADF8D939D9342
:100650000895CF93CFB7CF93DF93C395499BE9F725
:10066000499B0BC0499B09C0499B07C0499B05C0DA
:10067000499B03C0499B01C089C06F93C09122016F
:10068000DD27C75DDE4F2F9365E5499B03C02F91A2
:100690006F91E6CF0F931F934F9320E040E15F935C
:1006A00009B1067001FB27F93F9350E03BE039C0E8
:1006B000167040642F77012F5F5F1EC0406819B12C
:1006C00016702F7752501FC0406409B12F77067003
:1006D000D1F15F5F00C023C0406219B12F7716705F
:1006E00091F15F5F00C025C006701027515012F4D1
:1006F0005D5F0000115027952C3F19B1C8F61670A8
:100700000127015027952C3FC8F64227499309B18C
:10071000067010274F73115027952C3FA8F6469569
:10072000469519B1167079F00127015027952C3F95
:1007300098F66B5A60F3315009B1B0F600C011E081
:100740001CBB002717C03B503195C31BD04011E0A4
:100750001CBB0881033CF9F00B34E9F02091200127
:100760001981110F1213EDCF093651F10D3211F02D
:10077000013E39F7009327013F915F914F911F91FF
:100780000F912F916F91CCB3C0FD67CFDF91CF91C7
:10079000CFBFCF91189520912701222369F31091A3
:1007A0002501112339F534303AF130932501209396
:1007B0002101109122013BE0311B309322011CC02A
:1007C000009125010130B4F40AE53091000134FDB7
:1007D00014C000930001C5E1D1E013C0052710E06B
:1007E00000C000000BB91AC0052710E0221F1DC071
:1007F00010E021C04AE502C032ED432FC4E1D0E051
:1008000032E01AB11660599A0BB11AB956E020E8D5
:1008100065E320FF05270BB9279517951C3FF0F6D8
:100820006695B8F7B1F720FF05270BB927951795FF
:100830001C3FD0F62795179517FF052700001C3F92
:100840000BB9B0F629913A9519F7097F1091260155
:10085000110FC651D0400BB911F01093200111E0D7
:100860001CBB02601AB1197F402F497F54E05A9592
:10087000F1F70BB91AB94BB97FCFFB01A8953197A6
:100880008040E1F70895DC0113963C91139714968C
:10089000EC91149712962C911297203331F4E37057
:1008A000F0E0EE5FFE4F80810895932F8E2F283564
:1008B00049F4332391F4E1E0F0E089E080935700BC
:1008C000849108952035E1F4332389F4E0E0F0E0E9
:1008D00089E08093570084910895383009F036C03C
:1008E000E3E0F0E089E08093570084910895383088
:1008F00069F5E2E0F0E089E0809357008491089583
:10090000203251F4A0E0B0E0880F991FAA1FBB1F4E
:10091000ABBFFC0187910895283269F4A0E0B0E0F4
:10092000880F991FAA1FBB1F0196A11DB11DABBF48
:10093000FC0187910895203A09F46AC2203C21F411
:1009400015966C9172D202C02F3F11F080E008958D
:1009500081EF80930B0180E008951AB881E08BB994
:1009600085BF82E085BF60E071E787DF04B603FEE4
:100970000EC08EEF9FE054D210E0805B904B09F4E4
:1009800011E08EEF9FE06FEF7FEF5DD208C004B6FD
:1009900001FC02C010E003C019B11095117014BE23
:1009A000112309F427C28EEF80930B0114BE88E156
:1009B0000FB6F89480936000109260000FBE809193
:1009C0006900826080936900E89A519A8CE060E047
:1009D00075E353DF5198789481EF80930B019091E8
:1009E0002501935097FD52C180912201CCE0D0E0C7
:1009F000C81BD109C75DDE4F809121018D3209F0FE
:100A0000C2C0983009F040C183EC809315018AE59B
:100A10008093000110920A013881832F807629810A
:100A2000882309F441C086E091E0909324018093EB
:100A30002301233031F4CE0126DF8093090124E025
:100A400098C0253079F12A3069F1822F84508630A0
:100A5000E0F48A819B8190930D0180930C012930F1
:100A600039F48C819D8190930F0180930E0118C001
:100A70008E81809310018D8182708093110120936B
:100A8000120137FD71C09FEF70C0223021F48091B8
:100A90000B018E7F03C080910B01816080930B015D
:100AA00020E067C021E065C08A8110921E012223E8
:100AB00031F410921F018EE191E022E050C0253008
:100AC00019F48093260148C02630B1F58B8181301E
:100AD00019F48AED90EE04C0823041F48CEE90EE71
:100AE000909324018093230122E122C08330F9F402
:100AF0008A81882341F48CEA90EE909324018093BC
:100B0000230124E015C0813041F480EB90EE9093F6
:100B10002401809323012CE10BC0823041F48CEC42
:100B200090EE90932401809323012EE001C020E0F9
:100B300080E480930A011DC0283019F488E291E016
:100B400009C0293019F48093280106C02A3021F405
:100B50008EE191E021E003C08EE191E020E09093EE
:100B600024018093230105C09E8180E880930A01BF
:100B700007C08F81882319F49E81921708F0922F65
:100B80009093010181C080910A0187FF7DC080910F
:100B90001001092F891708F4082F801B809310017A
:100BA000FF24882311F4FF24F39410E066C08091A1
:100BB0001201873070F080910C0190910D01019627
:100BC00090930D0180930C01019769912ED11F5FC5
:100BD00054C040910C0150910D0160910E01709133
:100BE0000F01403080EE580781E0680780E0780709
:100BF00008F048C01E5FF8948991999121E00C019A
:100C0000FA0160935B0020935700E89511247894D3
:100C1000DB01CA010296A11DB11D80930C019093C6
:100C20000D01A0930E01B0930F01882341F0FF2026
:100C300021F1101710F1809111018823F1F0F8943F
:100C400083E0FA0160935B0080935700E895789405
:100C500007B600FCFDCFF89485E0FA0160935B00D5
:100C600080935700E895789407B600FCFDCFF89480
:100C700081E180935700E8957894101708F497CF96
:100C8000FF2011F0109201011092250180910001C6
:100C900084FF8CC0809101018F3F09F487C0182F19
:100CA000893008F018E0811B8093010180911501C3
:100CB00098E8892780931501112309F465C0809174
:100CC0000A0187FF3DC080911001811708F4182F99
:100CD000811B8093100100911201C6E1D1E028C070
:100CE000073030F080910C0190910D0191D00BC034
:100CF00080910C0190910D01A0910E01B0910F0116
:100D0000ABBFFC0187918883219680910C01909163
:100D10000D01A0910E01B0910F010196A11DB11D11
:100D200080930C0190930D01A0930E01B0930F01DD
:100D3000812F90E08A5E9E4FC817D90789F622C09E
:100D4000C0912301D091240186FF11C0212F46E1DB
:100D500051E0CE01A0E0B0E0A160ABBFFC01879103
:100D6000FA018193AF012196215099F707C0912F85
:100D7000E6E1F1E0899181939150E1F7D09324016C
:100D8000C0932301193060F486E191E0612F5DDCAE
:100D9000612F6C5F6C3041F08FEF8093010104C0D4
:100DA0008FEF809301016EE16093000194E189B1BE
:100DB000867031F49150D9F71092260110922001DB
:100DC00080910B01803130F0489B0FC080910B0166
:100DD000805109C0489909C080910B01823028F0E8
:100DE00080910B01825080930B0180910B0188232D
:100DF00009F0F5CDF894519A1BB81DBA109269000C
:100E000081E085BF15BEE0911301F09114010995B1
:100E1000F999FECF92BD81BDF89A992780B50895C2
:100E2000A8E1B0E042E050E013C0262FF999FECFD0
:100E30001FBA92BD81BD20BD0FB6F894FA9AF99AF7
:100E40000FBE01960895F1DF272FF0CFDC01CB0113
:100E5000FC01F999FECF06C0F2BDE1BDF89A3196CA
:100E600000B40D9241505040B8F70895F894FFCF68
:100E70005AFF1E970500DC0101C06D9341505040A0
:080E8000E0F70895F894FFCF9C
:020E8800CE0496
:00000001FF
